:020000040000FA
:100000008316F03086002730810083128B01033085
:100010008600831618308500831290012C309800DA
:1000200064309900920181010B110B1D1A28900A6E
:100030000B111D28000000000000980B15282C3023
:100040009800990B152883161030850083128511AE
:10005000010891000B19900A0B119601960A85155B
:100060000000851100000108110203192E289609CD
:10007000160A92000310900C910C920C0310900C35
:10008000910C920C013093005F3094009030061A6E
:10009000AE309500861A4E286B204F2860207620BF
:1000A00086100D08F0390319F0308D040D089F20DB
:1000B000861406100E089F200F089F20061409289A
:1000C0001508920714080318140F91071308031852
:1000D000130F90070800150892021408031C140F50
:1000E00091021308031C130F90020800031018302C
:1000F00097008F018E018D018C01920D910D900D55
:100100008F0D8E0D8D0D8C0D970B872800340F30C1
:10011000840094200E30840094200D3084009420BC
:100120000C30840094207D28033000079600961937
:100130008000303000079600961B80000034960047
:1001400008309700960D031886150615000000006C
:0E0150000000000006118611970BA22808007F
:02400E00F13F80
:00000001FF
